:1000000000308A0039290000831A0A28A500030E4F
:10001000A6000F288312A500030EA600A614A50EA5
:100020000408A7002008A8002108A9002208AA00A7
:100030002308AB002408AC0083128B1E21280B1967
:1000400044280B1E25288B183828270884002808E8
:10005000A0002908A1002A08A2002B08A3002C0850
:10006000A400260E83008312250EA618831609000D
:100070003208B4003108B300B201B1012E1440308F
:1000800087068B108A112528DB308100B10A0319FD
:10009000B20A3208273C03185B28FF3A031D542894
:1000A00031084B3C03185B28B201B1012E142830F3
:1000B000B4004B30B3000B118A112528941283161B
:1000C000871207168711003083129400831694005C
:1000D00083129001A1009200003083169200FF303D
:1000E0008600003087000108C03902388100831281
:1000F0008B160B16C0308B04831607118312071161
:100100000C3097000030A10004389200FF308316B5
:10011000920083129501B201B1013208B400310896
:10012000B300831681130117831240293B308400EA
:1001300000080319A9280330A100A001A00B9E28E4
:10014000A10B9D28E330A000A00BA4280000800B89
:100150009B2800340713BA01B9013A08033C031C79
:10016000D128031DB7283908FE3C031CD1283A08C2
:10017000A2003908A100A20CA10CA20CA10CA20C97
:1001800021089500A20C220C3039A0001708CF39A5
:10019000200497000130BB009620B90A0319BA0A5F
:1001A000AD2807170330BA00FF30B90039083A0408
:1001B0000319F5283A08A2003908A100A20CA10CE5
:1001C000A20CA10CA20C21089500A20C220C303923
:1001D000A0001708CF39200497000130BB009620FB
:1001E00039080319BA03B903D62807134329A00114
:1001F000A101A201A301C101C201C301C4014008C0
:100200003F043E043D04031935292030C500031086
:10021000B90DBA0DBB0DBC0DC10DC20DC30DC40D82
:1002200040084402031D1E293F084302031D1E29E6
:100230003E084202031D1E293D084102031C2F29CE
:100240003D08C1023E08031C3E0FC2023F08031CCA
:100250003F0FC3024008031C400FC4020314A00D4B
:10026000A10DA20DA30DC50B07290000413084008C
:100270005E2984011F30830583169F0183125E2847
:1002800086184329AA282E1C7E292E10B408031D87
:1002900050293308863C031C5029B4018730B30031
:1002A000BC010230BB001B30BA007930B900C0017C
:1002B000BF013408BE003308BD00F7282308B8008A
:1002C0002208B7002108B6002008B5003608B000A3
:1002D0003508AF002F08B90030080339BA00BA0C4E
:1002E000B90CBA0CB90CBA0C39089500BA0C3A0C16
:1002F0003039A0001708CF39200497004029630047
:02400E00020DA1
:00000001FF
